:020000040000FA
:10000000000005280000000000288312031385016A
:10001000043086004030870083163A308500CB30AC
:1000200086008030870006309F006400C430810065
:100030008312901010169016A001A0152015E92328
:100040007223851C4428A0148523BE21851C4428C6
:10005000A0148523EE21851C4428A0148523E620C6
:100060000511BE23851C4428A0148523FE1BE9230B
:10007000851C4428D422851C4428A0148523BE2135
:10008000851C4428172221284720202431280515C3
:1000900070200511003A03195128023A0319652806
:1000A000080024082102031C483E463C031C0800AB
:1000B000210884002A0880002108773C031D63285A
:1000C0003030A1000800A10A0800A010BE21851848
:1000D0006D28BE23A01D662808002A24FE01080002
:1000E00006300B24A010AA010830AF00A013201086
:1000F000A501851825140230102400308518013020
:100100002506031995280130102400308518013088
:10011000A500FE0A80302518FE050E307E06031964
:100120000234251801340000992801301024000001
:10013000892814300B2413300B24A50185182514AD
:100140000230102400308518013025060319BB2821
:1001500001301024003085180130A500250CAA0CB0
:10016000FE0A80302518FE050E307E060319023483
:10017000AF0B9928BF28013010240000AE2813309F
:100180000B2413300B2400000000A5018518251452
:100190000230102400308518013025060319E228AA
:1001A00001301024003085180130A500FE0A80308F
:1001B0002518FE050E307E060319E12825180034A7
:1001C00001340234013010240000D628A01E08009B
:1001D000A0190800A01F0800201F08002208A50081
:1001E0002808A600851C08000514A0130515220880
:1001F00084000008AB008C21003A031D392900005F
:100200002208FF3C031907290000A20A0A29A0308E
:10021000A2000000A80BF428A01225088400000802
:10022000A800210884002808851E1F2980002108B5
:10023000773C031D1E293030A1001F29A10A01307F
:10024000AD022508840000308000A60B30298618F6
:10025000080048302D02031C06117F1848290800A9
:100260002508FF3C03193629A50A0D29A030A50051
:100270000D29051481012508A2002608A800BE2129
:100280008A300102031C3F29201005102A2408008F
:10029000AB01E5307D2110307D2150307D21503083
:1002A0007D2101307D210030F81B0238F91B043814
:1002B000FA1B08387D2116307D2178087F397D2191
:1002C00079087F397D217A087F397D210030FB1B39
:1002D0000238FC1B0438FD1B08387D2132307D219B
:1002E0007B087F397D217C087F397D217D087F391E
:1002F0007D212B097D217F100800A500AB06210878
:100300008400250880002108773C031D8A293030AD
:10031000A1000800A10A0800000017300B2485186E
:10032000013419300B2400000830AF002B18A62927
:10033000000005141A300B248518013418300B24E2
:1003400000000310AB0CAF0B9629B32905101A302F
:100350000B24851C013418300B2400000310AB0C57
:10036000AF0B9629B32900000000051019300B24AB
:10037000851C0134000016300B24003460302D023F
:100380000319DC298C1ED8299818E1291819E629A7
:10039000AD0A4C302D0203180615230884001A08F4
:1003A00080002308FF3C031DDF29A030A3000800C4
:1003B0000000043010240800053010240800A30AAF
:1003C0000800181218160330102408001A08031920
:1003D000FE17013010240000ED290800861CF129C9
:1003E000152A0000201E092A8316981C102A0000D6
:1003F0008312240884000008990000308000A90BB3
:10040000022A20122408773C031D0E2A3030A40053
:10041000080004301024000000000800A40A0800AE
:10042000831203301024000008000000092A8618F7
:100430000800A01A080022082302031C603E0319CA
:100440003C2AA700AD008618292A48302D02031C3B
:10045000061122088400851C0800801B402A8001A8
:100460000408FF3C0319362A840A382AA030840085
:10047000A70B2B2A2308A200AD01861C0611080039
:100480000408A200001B4C2A801A492A0230A80046
:10049000632A0430A800632A801A512A0630A80073
:1004A000632A2708013C031808000408FF3C0319CD
:1004B0008A2A840A0008A800023C0318782A28081F
:1004C000203C031C782A851C08002808AF00A522C0
:1004D000003A03190800023A0319782A2808AF00E5
:1004E000AF038D22003A03197A2A023A0319080051
:1004F000BD220800851C0800CC22851E872A2408FE
:100500002102031C483E2807283C031C0800A016B3
:10051000AC010800A03084005A2A22088400000898
:10052000AB0000000408FF3C0319A22A840A00085B
:10053000AB06851C0234AF0B922A2B08FF3A031935
:1005400000340134A0308400972A2208840000007F
:10055000A92A23080402031900340408FF3C0319E4
:10056000B52A840AAF0BB82A0134A0308400B22A1D
:10057000801B0234851C0034A92A0030A800220800
:100580008400003080000408FF3C0319C92AA20A35
:100590000800A030A2000800220884000008813A68
:1005A000031D08007F140800201A080024082102F7
:1005B000031C483E03190800A70024088400851C7A
:1005C0000800801BF12A80010408773C0319EA2AFD
:1005D000840AEC2A30308400A70BDF2A2108A4000B
:1005E00008000408A400001BFD2A801AFA2A023021
:1005F000A900142B0430A900142B801A022B0630FA
:10060000A900142B2708013C031808000408773CB4
:1006100003192F2B840A0008A900023C0318292B78
:100620002908203C031C292B851C08002908AF0041
:100630004A23003A03190800023A0319292B290812
:10064000AF00AF033223003A03192B2B023A0319F0
:10065000080062230800851C0800201608003030BE
:1006600084000B2B2408840000080000A500040867
:10067000773C0319472B840A0008A506851C023421
:10068000AF0B372B2508FF3A031900340134303003
:1006900084003C2B2408840000004E2B2108040217
:1006A000031900340408773C03195A2B840AAF0B52
:1006B0005D2B013430308400572B801B0234851CA5
:1006C00000344E2B0030A900240884000030800044
:1006D00030240408773C03196F2BA40A080030303B
:1006E000A40008009817831618129816181583127C
:1006F0004B30051E7F2B403085197F2B143083161D
:1007000099008312181606110800A01B942B201CB8
:10071000902BBA300102031C08002010A01708001B
:100720008101201320140800201B0800201CB52B79
:1007300003308A002C082C07820700000000BA3022
:10074000AF2BA730AF2B9430AF2B8130AF2B6E3057
:10075000AF2B5B30AF2B4930AF2B3630AF2B0102C4
:10076000031C0800201020170800A01EAC012C0854
:10077000083A031DAC0A810120140800A019CF2BF0
:10078000A0181010101CCA2B0C1C08001010A0156B
:10079000201508008E018F010C1010140800201D78
:1007A000D32BA01C08002019DE2B0C1C0800A60B64
:1007B000E72B101010169016A0110800201105301C
:1007C000A600E923101290168E018F0110140C1050
:1007D0000800F801F901FA01FB01FC01FD01FE012D
:1007E000AD012012A0127F10AC01A030A300A20026
:1007F000840080010408FF3C0319002C840AF92BB3
:100800003030A100A400840080010408773C031963
:100810000800840A042C10240000BE21EE210800E8
:10082000AE00AE0B112C0800851D142C05301024D1
:100830008519182C0530102405110800FF3EFF3ED5
:100840001230A500000005301024851C0800A50BFF
:10085000232C0800FD0F0800FC0F0800FB0A08000D
:0C086000FA0F0800F90F0800F80A080061
:084000000100060003000200AC
:02400E00F23F7F
:00000001FF
